:020000040800F2
:10000000000001200D620008855A00088B5A000884
:10001000915A0008975A00089D5A000800000000F5
:1000200000000000000000000000000091D7000860
:10003000A35A00080000000081D80008AF5A000849
:1000400055620008556200085562000855620008B4
:1000500055620008C95A0008556200085562000838
:100060005562000855620008556200085562000894
:100070005562000855620008556200085562000884
:100080005562000855620008556200085562000874
:100090005562000855620008556200085562000864
:1000A0005562000855620008556200085562000854
:1000B00055620008D55A00085562000855620008CC
:1000C0005562000855620008556200085562000834
:1000D0005562000855620008556200085562000824
:1000E00055620008556200085562000800000000D3
:1000F0000000000000000000000000000000000000
:100100000000000000000000556200085562000871
:1001100055620008556200085562000855620008E3
:1001200055620008556200085562000855620008D3
:1001300055620008E95A0008556200085562000837
:1001400055620008556200085562000855620008B3
:10015000000000000000000000000000000000009F
:10016000000000000000000000000000000000008F
:10017000000000000000000000000000000000007F
:10018000000000000000000000000000000000006F
:10019000000000000000000000000000000000005F
:1001A000000000000000000000000000000000004F
:1001B000000000000000000000000000000000003F
:1001C000000000000000000000000000000000002F
:1001D000000000000000000000000000000000001F
:0401E0005FF8E0F1F3
:1001F00010B5054C237833B9044B13B10448AFF361
:1002000000800123237010BDB80000200000000012
:100210005CDB010808B5034B1BB103490348AFF38E
:10022000008008BD00000000BC0000205CDB01086D
:1002300010F8012B11F8013B012A28BF9A42F7D090
:10024000D01A7047034613F8012B002AFBD1181A65
:100250000138704753B94AB9002908BF00281CBFAC
:100260004FF0FF314FF0FF3000F076B9ADF1080CE0
:100270006DE904CE00F006F8DDF804E0DDE90223C4
:1002800004B070472DE9F047089E0D4604468846A5
:10029000002B4DD18A42944668D9B2FA82F252B10B
:1002A00001FA02F3C2F1200120FA01F10CFA02FC7A
:1002B00041EA030894404FEA1C41B8FBF1F71FFAEA
:1002C0008CFE01FB178807FB0EF0230C43EA084362
:1002D00098420AD91CEB030307F1FF3580F01E8119
:1002E000984240F21B81023F63441B1AB3FBF1F0BA
:1002F00001FB103300FB0EFEA4B244EA0344A64502
:100300000AD91CEB040400F1FF3380F00981A645F3
:1003100040F20681644402380021A4EB0E0440EA56
:1003200007401EB10023D440C6E90043BDE8F08772
:100330008B4208D9002E00F0EE800021C6E90005AE
:100340000846BDE8F087B3FA83F100294AD1AB42F1
:1003500002D3824200F2FC80841A65EB0303012081
:100360009846002EE2D0C6E90048DFE702B9FFDE7A
:10037000B2FA82F2002A40F09180A1EB0C00012138
:100380004FEA1C471FFA8CFEB0FBF7F307FB130084
:10039000250C45EA00450EFB03F0A84208D91CEBEA
:1003A000050503F1FF3802D2A84200F2CE80434691
:1003B0002D1AB5FBF7F007FB10550EFB00FEA4B29B
:1003C00044EA0544A64508D91CEB040400F1FF35B6
:1003D00002D2A64500F2B6802846A4EB0E0440EAFD
:1003E00003409EE7C1F120078B4022FA07FC4CEA4C
:1003F000030C25FA07FA4FEA1C49BAFBF9F820FA70
:1004000007F309FB18AA8D401FFA8CFE1D4300FA62
:1004100001F308FB0EF02C0C44EA0A44A04202FA55
:1004200001F20BD91CEB040408F1FF3A80F088803C
:10043000A04240F28580A8F102086444241AB4FB6B
:10044000F9F009FB104400FB0EFEADB245EA04448E
:10045000A64508D91CEB040400F1FF356CD2A64573
:100460006AD90238644440EA0840A0FB0295A4EB34
:100470000E04AC42C846AE4656D353D0002E69D0C7
:10048000B3EB080264EB0E0422FA01F304FA07F757
:100490001F43CC40C6E90074002147E70CFA02FC78
:1004A000C2F1200125FA01F34FEA1C4720FA01F1BD
:1004B00095400D43B3FBF7F107FB11331FFA8CFE98
:1004C000280C40EA034001FB0EF3834204FA02F4D5
:1004D00008D91CEB000001F1FF382FD283422DD93F
:1004E00002396044C01AB0FBF7F307FB1300ADB24A
:1004F00045EA004503FB0EF0A84208D91CEB0505B0
:1005000003F1FF3816D2A84214D9023B6544281AD9
:1005100043EA014138E73146304607E72F46E4E633
:100520001846F9E64B45A9D2B9EB020865EB0C0E6B
:100530000138A3E74346EAE7284694E74146D1E776
:10054000D0467BE76444023847E7023B65442FE727
:10055000084606E73146E9E6704700BF80B485B03B
:1005600000AF78600B467B804DF27F73FB817B8808
:100570005A1E7A80002B14BF01230023DBB2002B0C
:1005800025D07B685A1C7A601B781B021AB2B7F917
:100590000E3053401BB2FB810023BB60BB68072BAE
:1005A000E5DCB7F90E30002B0ADAFB895B00FB8132
:1005B000FB8983F4FF4383F07A03DB43FB8102E092
:1005C000FB895B00FB81BB680133BB60E6E7FB890D
:1005D00018461437BD4680BC704780B586B000AF62
:1005E000F8600B467A607B817B89072B01D800235A
:1005F00052E0FB681B78FD2B01D000234CE0FB6828
:1006000001331B781B021AB2FB6802331B781BB242
:1006100013431BB29BB2033B9AB27B681A817B687F
:100620001B8903F108027B899A4201D0002333E041
:100630007B89023BFA6813441B781B021AB27B8940
:10064000013BF9680B441B781BB213431BB2FB82BE
:100650007B89023B9BB21946F868FFF77FFF034690
:100660001A46FB8A934214BF01230023DBB2002BFE
:1006700001D0002310E0FB68DA787B685A70FB68D1
:100680001A797B681A70FB685A797B689A70FB68E4
:100690009A1D7B685A60012318461837BD4680BDF5
:1006A00080B483B000AF78607B6800221A817B68D9
:1006B00018460C37BD4680BC704780B586B000AF89
:1006C000F860B96011461A460B46FB8013467B71F1
:1006D000FB681B89DA1DFB889A4201DB00238AE054
:1006E000BB68FD221A70FB681B8903331A12BB68B2
:1006F0000133D2B21A70FB681B89DAB2BB680233CD
:100700000332D2B21A70BB680333FA6852781A7097
:10071000BB680433FA6812781A70BB680533FA684C
:1007200092781A70FB681B89002B08D0BB68981D53
:10073000FB685968FB681B891A461BF0D7FDFB68EC
:100740001B8906339BB21946B868FFF707FF0346BB
:100750007B827B8A1B0A99B2FB681B890633BA68C5
:100760001344CAB21A70FB681B890733BA68134472
:100770007A8AD2B21A70FB681B890833FB827B79B4
:10078000002B37D00123BB82BA8AFB8A9A4231D22E
:10079000BB8ABA6813441B78FC2B05D0BB8ABA68A5
:1007A00013441B78FD2B21D1BB8A0133BA68D018C2
:1007B000BB8ABA68D118FA8ABB8AD31A1A461BF0C8
:1007C000A3FDBA68BB8A591CB9821344FC221A7073
:1007D000BB8ABA6813441A78BB8AB9680B4402F022
:1007E0007F02D2B21A70FB8A0133FB82BB8A0133CB
:1007F000BB82C9E7FB8A18461837BD4680BD00009A
:1008000080B584B000AF7860154B1B785A1C154B2F
:1008100083FB02139910D317C91A0B465B000B44D4
:10082000DB00D11ACAB20E4B1A700023FB73FB7B9C
:10083000022B11D8FB7B0C4A52F82330002B0AD034
:10084000FB7B094A52F82330184600F0BFF8FB7BC7
:100850000133FB73EBE700BF7D200BF0EDFED3E728
:10086000D4000020ABAAAA2AD800002080B582B00C
:1008700000AF786039600E4A3B681360786804F016
:100880001CFE024613461B029B1A0A4A13600A4BBF
:100890001B68002B07D1094A002109480AF01CF9FE
:1008A0000346054A136000BF0837BD4680BD00BF40
:1008B000E8000020EC000020E4000020000F020807
:1008C0000108000880B485B000AF78600B467B80DB
:1008D0000023FB73FB7B022B12D8FB7B0B4A52F8E5
:1008E0002330002B08D1FB7B08497A6841F823208C
:1008F0007B687A885A8003E0FB7B0133FB73E9E76E
:100900007B6818461437BD4680BC7047D80000206D
:1009100080B582B000AF78600B46FB707B68FA78D8
:100920001A70786800F052F800BF0837BD4680BDE5
:1009300080B483B000AF78600B46FB707B685B8847
:10094000002B0CD1FB78002B03D01E4B1B681A46E2
:1009500000E000221C4B1B681B685A632DE07B687B
:100960005B88042B0CD1FB78002B03D0154B1B6844
:100970001A4600E00022144B1B681B689A631CE0B7
:100980007B685B88082B0CD1FB78002B03D00D4BC8
:100990001B681A4600E000220B4B1B681B68DA63D9
:1009A0000BE0FB78002B03D0064B1B681A4600E0D7
:1009B0000022054B1B681B681A6400BF0C37BD463C
:1009C00080BC7047EC000020E800002080B582B0B9
:1009D00000AF78607B681B78052B4FD801A252F8D6
:1009E00023F000BFFD090008070A0008110A0008EB
:1009F0002D0A0008490A0008650A000800217868E5
:100A0000FFF796FF3AE001217868FFF791FF35E0A4
:100A10001C4B1B7803F00403002B0CBF01230023A5
:100A2000DBB219467868FFF783FF27E0154B1B7888
:100A300003F00403002B14BF01230023DBB219468B
:100A40007868FFF775FF19E00E4B1B7803F0010380
:100A5000002B0CBF01230023DBB219467868FFF797
:100A600067FF0BE0074B1B780B2B94BF0123002380
:100A7000DBB219467868FFF75BFF00BF00BF08379D
:100A8000BD4680BDD400002080B483B000AF786044
:100A90007B6800229A607B6818460C37BD4680BC94
:100AA000704780B483B000AF78607B689B68002B90
:100AB0000CBF01230023DBB218460C37BD4680BCB7
:100AC000704780B582B000AF786039607B681846A7
:100AD000FFF7DAFF386800F03CF80346002B0DD032
:100AE0003B689B6878683968022298473B68DA68F7
:100AF0007B68DA603B689A687B689A607B68184616
:100B00000837BD4680BDF0B585B000AFF860B9606C
:100B10001346FB80FB681846FFF7C3FF0346002B14
:100B200001D01BF07AFAFB68DC68FD6807F1080366
:100B3000184600F01EF80646BB1D184600F023F8C4
:100B400003461A4631462846A04700BF1437BD4623
:100B5000F0BD80B582B000AF78607B681846FFF7C3
:100B6000A0FF034683F00103DBB218460837BD46F9
:100B700080BD80B483B000AF78607B6818460C37C6
:100B8000BD4680BC704780B483B000AF78607B689E
:100B900018460C37BD4680BC7047000080B400AFDB
:100BA000BFF34F8F00BF064BDB6803F4E0620449DC
:100BB000044B1343CB60BFF34F8F00BF00BFFDE773
:100BC00000ED00E00400FA05B0B594B000AF07F105
:100BD00018033822002118461BF0B0FB0123BB612B
:100BE0004FF480333B6204237B620123FB624FF4AA
:100BF0008033FB610223BB634FF48033FB634FF40C
:100C0000E0133B6402237B644FF4C063BB64402366
:100C1000FB6407F11803184607F0B4F90346002BEC
:100C200014BF01230023DBB2002B01D000F0DEFC57
:100C3000114B3C1D1D460FCD0FC42B6823603B1D7F
:100C40000221184607F0B4FC0346002B14BF012311
:100C50000023DBB2002B01D000F0C8FC00224FF0D3
:100C6000C061002007F08EFD044B01221A6000BF16
:100C70005037BD46B0BD00BF84DB01087000424262
:100C800080B58EB000AF554B554A1A60534B0022C9
:100C90005A60524B00229A60504B4FF6FF72DA6056
:100CA0004E4B00221A614D4B00229A614B4807F0CF
:100CB000CFFE0346002B14BF01230023DBB2002B21
:100CC00001D000F093FC07F1280300221A605A605B
:100CD0009A60DA604FF48053BB6207F1280319462B
:100CE0003E4808F0CDF90346002B14BF0123002332
:100CF000DBB2002B01D000F079FC384807F0F7FE9A
:100D00000346002B14BF01230023DBB2002B01D0CC
:100D100000F06CFC00233B6200237B6207F12003A0
:100D200019462E4808F04CFD0346002B14BF012342
:100D30000023DBB2002B01D000F058FC3B1D002249
:100D40001A605A609A60DA601A615A619A61602387
:100D50007B600223FB603B1D002219461F4808F000
:100D6000D1F80346002B14BF01230023DBB2002B74
:100D700001D000F03BFC3B1D04221946174808F047
:100D8000C1F80346002B14BF01230023DBB2002B64
:100D900001D000F02BFC3B1D082219460F4808F03B
:100DA000B1F80346002B14BF01230023DBB2002B54
:100DB00001D000F01BFC094804F086FD0021074823
:100DC00007F0EEFE0421054807F0EAFE082103487B
:100DD00007F0E6FE00BF3837BD4680BDF0000020BA
:100DE0000004004080B500AF134B144A1A60124B48
:100DF0004FF4E1325A60104B00229A600E4B0022F1
:100E0000DA600D4B00221A610B4B0C225A610A4B1F
:100E100000229A61084B0022DA61074808F048FD79
:100E20000346002B14BF01230023DBB2002B01D0AB
:100E300000F0DCFB00BF80BD38010020003801401D
:100E400080B588B000AF424B9B69414A43F0100324
:100E500093613F4B9B6903F01003FB60FB683C4BC5
:100E60009B693B4A43F020039361394B9B6903F034
:100E70002003BB60BB68364B9B69354A43F00403D3
:100E80009361334B9B6903F004037B607B68304BB9
:100E90009B692F4A43F0080393612D4B9B6903F034
:100EA00008033B603B68002242F23021294807F0EA
:100EB00050F8002240F20721274807F04AF80122A3
:100EC00044F24001244807F044F807F110030022DF
:100ED0001A605A609A60DA6042F230233B61012363
:100EE0007B610023BB610223FB6107F110031946FC
:100EF000184806F093FE01233B6100237B61012328
:100F0000BB6107F110031946124806F087FE44F250
:100F100047233B6101237B610023BB610223FB610B
:100F200007F1100319460C4806F078FE4FF4807361
:100F30003B6102237B610223FB6107F11003194629
:100F4000064806F06BFE00BF2037BD4680BD00BFDF
:100F50000010024000100140000C01400008014058
:100F600080B582B000AF7860094B93F83B309B109E
:100F7000DBB203F00103002B01D0064B00E0064B6F
:100F8000194606481BF0BEFA00BF0837BD4680BDB3
:100F9000740A002098DB01089CDB0108A4DB01082F
:100FA00080B500AF00224FF48041084806F0D1FF21
:100FB000322005F0B3F901224FF48041034806F0D6
:100FC000C8FFFA2005F0AAF900BF80BD000C01405F
:100FD00080B584B000AF3B4600221A605A609A6028
:100FE000DA6008233B6001237B600023BB6002239F
:100FF000FB603B461946074806F010FE0022082118
:10100000044806F0A6FFFFF7CBFF00BF1037BD4630
:1010100080BD00BF0008014080B588B000AFF86017
:10102000B9607A603B6001212B4806F07BFF0346E4
:10103000002B0CBF01230023DBB2002B48D0022180
:10104000B868FFF765FC0023FB7705F05DF9B86130
:101050004FF47A73FB8201211F4806F063FF0346B9
:10106000002B0CBF01230023DBB2002B2CD005F09A
:101070004BF938613A69BB69D21AFB8A9A42EAD9BC
:10108000FB7F0133FB773B69BB61FB7F032B03D9FC
:101090000421B868FFF73CFCFB7F062BDBD900215D
:1010A000B868FFF735FC01213868FFF731FC0121F2
:1010B0007868FFF72DFCF86804F072F94FF4FA70C5
:1010C00005F02CF9FFF76AFD0021B868FFF720FC56
:1010D00000BF2037BD4680BD0010014080B483B002
:1010E00000AF7860044A7B681A607B6818460C374A
:1010F000BD4680BC704700BF500F020880B582B06B
:1011000000AF78607B681846FFF7E8FF134A7B68FA
:101110001A607B68043300221A605A60C3F8072003
:101120007B6800221A617B6800225A617B68183351
:101130001E22002118461BF001F97B68363300217E
:101140000A461A800A469A707B68002283F8392082
:101150007B6818460837BD4680BD00BF840F020873
:1011600090B5CDB002AF07F59473A3F592731860F4
:1011700097481BF061FA07F18403184604F066F8FB
:1011800007F1840207F180031146184605F000F8C4
:1011900007F17C0300211846FFF794FB07F1780361
:1011A00004211846FFF78EFB07F174030821184647
:1011B000FFF788FB07F1840386491846FFF756FBC3
:1011C00007F17C0300211846FFF7A2FB07F1780323
:1011D00000211846FFF79CFB07F174030021184615
:1011E000FFF796FB07F1740307F1780207F17C0122
:1011F00007F18400FFF710FF07F17803022118467A
:10120000FFF786FB74481BF017FAFFF7E1FE07F1C2
:101210008403184608F0F2FE704B93F83B309B10A5
:10122000DBB203F00103002B02D16D481BF004FA7E
:1012300007F18403184604F0E3F8034619466948A9
:101240001BF060F968481BF0F7F907F17C0307F120
:10125000740207F1780107F1680000F0E3FF07F17D
:101260006803184601F028F860481BF0E5F9604B68
:101270001B68184600F0D4FE07F18403184604F0FA
:10128000BFF84FF4167301935023009302230022FA
:10129000584900F0B7FB07F18403184604F0B0F892
:1012A0004FF4167301934FF43C6300930323002221
:1012B000514900F0A7FB07F18403184604F0A0F899
:1012C0004FF4167301937B230093032300224B49B1
:1012D00000F098FB4A481BF0AFF907F114031846D9
:1012E000FFF70CFF07F114034649184601F081FF90
:1012F00007F1680207F114031146184601F086FF52
:1013000007F11403184602F04AFF034687F8233119
:1013100097F82331002B00F0898097F82331042BB4
:1013200009D0042B0FDC012B09D0032B0BD136483D
:101330001BF082F90BE035481BF07EF907E03448DA
:101340001BF07AF903E033481BF076F900BF07F190
:101350001403184602F0ECFE034619462E481BF013
:10136000D1F807F11403184602F003FF03461946AB
:101370002A481BF0C7F807F11403184602F0E3FEF1
:101380000346194626481BF0BDF807F1140318461A
:1013900002F0E4FE0346194622481BF0B3F807F1B9
:1013A0001403184602F0F0FEC7F81C01D7F81C31F0
:1013B0001B781946D7F81C3101331B781A46D7F829
:1013C0001C3102331B7818481BF09CF831E000BF39
:1013D000C0DB0108F0000020D4DB0108740A002003
:1013E000E4DB0108FCDB01080CDC01082CDC010853
:1013F000F8AD00203CDC010844DC010850DC0108A9
:1014000058DC01083801002078DC010894DC010870
:10141000ACDC0108C4DC0108E4DC0108F4DC0108F0
:1014200004DD010820DD01083CDD010866481BF0F1
:1014300069F807F16803184600F0AAFF63481BF03B
:10144000FBF807F1680207F110031146184603F094
:1014500011F807F11003184603F0B8FA5C481BF0C6
:10146000EBF807F11403184602F083FE044607F177
:101470001403184602F088FE024607F18003214655
:10148000184604F095FE07F18403184603F0C3FFE5
:101490000346002B0CBF01230023DBB2002B07D037
:1014A0004C4819F04FFD034619464B481BF02AF8EB
:1014B00007F1780300211846FFF72AFA07F17403B1
:1014C00002211846FFF724FA44481BF0B5F84FF004
:1014D000FF33C7F8243107F18403184603F0EDFF0A
:1014E0000246D7F82431934214BF01230023DBB214
:1014F000002B0CD007F18403184603F0DEFFC7F879
:10150000240107F1840336491846FFF7AFF94FF479
:101510007A700BF091F807F10C031A46012131485B
:1015200005F051FC0346002B0CBF01230023DBB266
:10153000002BD0D007F59473A3F58E731B6803F0CE
:101540000403002B1FD1284B93F83B309B10DBB2D8
:1015500003F00103002BBED007F18403184603F00B
:101560005AFF0346012B0CBF01230023DBB2002BE3
:1015700002D01D4816F056FD1B480EF035FE1A48E5
:101580000EF08AFEA7E7184B93F83B309B10DBB2B6
:1015900003F00103002B9ED113480EF04FFE1248BA
:1015A0000EF0CCFD07F18403184603F034FF034628
:1015B000012B0CBF01230023DBB2002B8BD00A4888
:1015C00016F054F887E700BF5CDD010880DD0108F4
:1015D0009CDD0108780A0020ACDD0108BCDD0108B3
:1015E000F000002020530020740A002080B400AFD7
:1015F00072B600BFFEE7000080B500AF04F02CFE1D
:10160000FFF7E2FAFFF71CFCFFF7ECFB0B4803F0D7
:10161000A7FCFFF735FB0A4B1B684FF6FF729A6376
:1016200009F0CCF9074A0021074809F055FA0346AA
:10163000064A136009F0F4F9FEE700BF3801002004
:10164000F0000020240F0208611100087C01002036
:1016500080B586B000AFF860B9607A60BB685A1C8C
:10166000BA601B783B613B6903F0C003C02B16D105
:101670003B691B0203F47C533B61BB685A1CBA6094
:101680001B781A463B6913433B613B69FA68134474
:101690007A681946F868FFF7DBFFBB682EE03B6904
:1016A00003F0C003002B05D0396916481AF02AFF51
:1016B000BB6823E000237B610AE0BA68531CBB606F
:1016C0007B68591C796012781A707B6901337B61E1
:1016D0007A693B699A42F0DB3B69002B05D17B6854
:1016E0005A1C7A6000221A7004E07B685A1C7A60E7
:1016F0002E221A703B69002BB0DCBB6818461837E5
:10170000BD4680BDD4DD010880B58AB000AFF86069
:10171000B9607A6000233B620023FB613B6ABB61D6
:1017200002E03B6A01333B623B6AFA6813441B7870
:101730002E2B05D03B6AFA6813441B78002BF0D19E
:101740003A6ABB69D31A7B61FB695A1C7B691344F3
:101750007A689A4209DAFB695A1C7B691344194674
:101760001B481AF0CFFE00232EE0BB685A1CBA605B
:101770007A69D2B21A70FB690133FB6100237B6284
:101780000DE0BA697B6A13441A46FB681A44BB68C9
:10179000591CB96012781A707B6A01337B627A6ACD
:1017A0007B699A42EDDBFA697B691344FB613B6A12
:1017B000FA6813441B782E2B02D13B6A01333B623B
:1017C0007B69002BAADCFB6918462837BD4680BD23
:1017D000F4DD010880B586B000AFF860B9607A60CA
:1017E0003B607A68B968F868FFF732FFB860BB6899
:1017F0001B683B613B8A18460DF04AFE03461A46B9
:101800003B6A1A807B8A18460DF042FE0346FB8233
:10181000FB8ADB0B9BB2DAB27B6A1A70FB8AC3F3DA
:101820000E039AB23B681A80BB6804331846183717
:10183000BD4680BD80B588B000AFF8607A603B607F
:101840000B467B81F868FEF7FDFC03460133FB6124
:101850003A8DFB6913441033BB61BB6918461AF01B
:1018600025FD03467B617B69002B04D1B9691648CD
:101870001AF048FE23E07B697A899A807B697A684E
:101880009A60FB699AB27B699A817B693A8DDA81A9
:101890007B691033FA69F96818461AF027FDFB696D
:1018A00010337A6913443A8D396818461AF01EFDD0
:1018B000064B1A687B691A60044A7B69136000BF93
:1018C0002037BD4680BD00BF18DE0108840100201E
:1018D00080B598B002AFF860B9607A6007F1140380
:1018E000402219467868FFF70FFF03467B657B6D42
:1018F000002B0AD07B6D9BB207F1140200931346B4
:10190000BA680C21F868FFF795FF00BF5837BD464D
:1019100080BD80B59AB002AFF860B9603B601346F5
:10192000FB800023BB820023FB82FB8818460DF05E
:10193000AFFD03463B8307F11403063340221946EB
:101940003868FFF7E1FEF865FB6D002B0CDDFB6DE1
:101950009BB206339BB207F1140200931346BA6898
:101960002121F868FFF766FF00BF6037BD4680BDE4
:1019700080B588B002AFF860B9607A607868FEF729
:1019800061FC0346FB82FB8AFF2B05D9FB8A1946C3
:1019900012481AF0B7FD1EE0FB8A013318461AF010
:1019A00085FC03463B61FB8ADAB23B691A703B69EE
:1019B0000133FA8A796818461AF098FCFB8A0133D9
:1019C0009BB200933B69BA681021F868FFF732FFB9
:1019D00038691AF073FC1837BD4680BD44DE010833
:1019E00080B586B002AFF860B9607A6004230093D6
:1019F0007B68BA680121F868FFF71CFF00BF103749
:101A0000BD4680BD80B58EB002AFF860B9607A6027
:101A1000FB70B868FEF716FC03460C33FB62FB6AEA
:101A2000013318461AF042FC0346BB62F868FEF721
:101A300009FC0246FB6A134401337B627B6A013373
:101A400018461AF033FC03463B62F868FEF7FAFBCF
:101A500003460733FB61FB69013318461AF026FC85
:101A60000346BB61FB6A591CFB7803F00103002BA2
:101A700001D0264B00E0264B0093BB68254AB86A8C
:101A80001AF094FF7B6A591CBB6A0093FB68224AD8
:101A9000386A1AF08BFFFB69591CFB681F4AB8694A
:101AA0001AF084FF7B68002B04D07A68F96B386ADF
:101AB000FFF75EFF00237B6107F114031A46F96B01
:101AC000B869FFF78DFF3A8FBB69F96B386AFFF78A
:101AD00020FF3A6AF96BB86AFFF7FAFEFB7803F069
:101AE0000203002B04D0BA6AF96B0D48FFF7F0FE31
:101AF000B86A1AF0E3FB386A1AF0E0FBB8691AF02A
:101B0000DDFB00BF3037BD4680BD00BF64DE01088D
:101B10006CDE010874DE010884DE01088CDE010839
:101B200098DE010880B584B000AF78600B467B80FA
:101B3000104B1B68FB6013E0FB689B887A889A4215
:101B400002D07B88FF2B08D1FB68103379681846D8
:101B50001AF0C4FF0346002B06D0FB681B68FB602D
:101B6000FB68002BE8D100E000BFFB681846103787
:101B7000BD4680BD8401002080B58AB000AFF8600A
:101B8000B9607A607B68C3F5A0737B62FB6803F180
:101B900010007B68BA6813447A6A1946FFF7B4FDEF
:101BA00003463B623B6A002B01D17B6854E0FB6833
:101BB000DB891A463B6A13440A337A6A9A420BD28B
:101BC000FB68DB891A463B6A13440A3319462448EA
:101BD0001AF098FC7B683FE07A683B6A13447B60AC
:101BE000FB689B8818460DF053FC0346BB8201201E
:101BF0000DF04EFC0346FB82FB689B6818460DF017
:101C000054FC0346BB61FB68DB8918460DF040FCC1
:101C10000346BB837B68BA6813441A4607F1140372
:101C200003CB106051601B8813817B680A337B6093
:101C30007B68BA68D018FB689B891033FA68D118A2
:101C4000FB68DB891A461AF051FBFB68DB891A46F0
:101C50007B6813447B607B6818462837BD4680BD8F
:101C6000B8DE010880B58AB002AFF860B9607A606A
:101C70007B689BB20022194600200EF09DFBF861A4
:101C8000FB69002B25D0FB695B687A68B968184648
:101C90001AF02CFB134BBB61134B5B687B61134B3E
:101CA00018687B69009341F2E943BA69F96914F055
:101CB00059FF0346FB7497F91330002B05D097F9B1
:101CC000133019460A481AF01DFCF8690EF0ECFEB4
:101CD00003E0796807481AF015FC00BF2037BD46BD
:101CE00080BD00BF540F0208C8650020800100209D
:101CF000E0DE0108FCDE010880B5B4B002AF786018
:101D000039603B68C7F8B4304FF4A0701AF0CEFACF
:101D10000346C7F8B030D7F8B030002B05D14FF4E8
:101D2000A07199481AF0EEFB2AE1D7F8B030C7F855
:101D3000AC303B681B889AB2D7F8AC301A80D7F821
:101D4000AC3084229A70D7F8AC300022DA70D7F821
:101D5000AC3000221A7100225A71D7F8AC30002240
:101D60009A710022DA71D7F8AC3000221A72002280
:101D70005A72D7F8AC3000229A720022DA720C2321
:101D8000C7F8C0300023C7F8BC30D7F8B4300C33E4
:101D9000C7F8B8303B689B889BB218460DF078FBBB
:101DA0000346C7F8A8300023C7F8C43092E007F113
:101DB000920107F10C0207F18F03019307F19003E1
:101DC00000930B46D7F8B810D7F8B400FFF702FD20
:101DD000C7F8B800B7F89230012B03D0B7F89230AB
:101DE000FF2B72D1B7F8902007F10C03114618466B
:101DF000FFF798FEC7F89C00D7F89C30002B64D002
:101E0000D7F89C309B88012B0FD1604B5B68C7F8DB
:101E10009830D7F89C309B891033D7F89C20134416
:101E2000D7F89820043212681A60D7F8C020D7F883
:101E3000B010D7F89C00FFF79FFE0346C7F8943018
:101E4000D7F8C030D7F894209A4215D9D7F8AC30DB
:101E5000DB889BB218460DF01BFB034601339BB297
:101E600018460DF015FB03461A46D7F8AC30DA8059
:101E7000D7F89430C7F8C030B7F890300C2B10D199
:101E8000D7F89C301B68002B1FD0D7F89C301B68FC
:101E90009B88212B19D1D7F89C301B68C7F8BC3020
:101EA00013E0B7F89030212B0FD1D7F89C301B6886
:101EB000002B0AD0D7F89C301B689B88012B04D1DB
:101EC000D7F89C301B68C7F8BC30D7F8C430013352
:101ED000C7F8C430D7F8C420D7F8A8309A42FFF624
:101EE00066AFD7F8C0300C2B46DDD7F8BC30002BDE
:101EF0003BD0D7F8BC309B88012B0FD1234B5B68BC
:101F0000C7F8A430D7F8BC309B891033D7F8BC2071
:101F10001344D7F8A420043212681A60D7F8C020FE
:101F2000D7F8B010D7F8BC00FFF726FE0346C7F875
:101F3000A030D7F8C030D7F8A0209A4215D9D7F8EA
:101F4000AC305B899BB218460DF0A2FA0346013310
:101F50009BB218460DF09CFA03461A46D7F8AC30EF
:101F60005A81D7F8A030C7F8C030D7F8C020D7F8CA
:101F7000B0107868FFF776FED7F8B0001AF09EF937
:101F8000C837BD4680BD00BF20DF0108C8650020FE
:101F900080B588B000AFF860B9607A603B607B685C
:101FA0001B89FB61FB69B3F5A07F30DCFB691B2B50
:101FB0002DDDFB6918461AF079F90346BB61BB6950
:101FC000002B04D1F96915481AF09CFA1FE0FB694F
:101FD0009AB20023B96978680EF070FF03461A467A
:101FE000FB69934210D1BB697B617B699B7803F0ED
:101FF000FA03002B08D17B699B889BB2002B03D08E
:1020000079693868FFF778FEB8691AF057F9786887
:102010000EF04AFD00BF2037BD4680BD44DF0108F9
:1020200080B584B000AF78607B68002B37D07B68C8
:1020300093F83B3003F02003002B1FD17B6893F80B
:102040003B3043F02003DAB27B6883F83B207868AA
:1020500017F088FF0346FB7397F90F30002B0DD064
:102060007B6893F83C3019467B6893F83D301A46FC
:1020700097F90F3024481AF045FA41E0234978686F
:1020800018F0D6F80346FB7397F90F30002B06D0F3
:1020900097F90F3019461E481AF034FA30E07B6881
:1020A000002B03D11B481AF0C7FA29E02E2014F0A8
:1020B0007DFF0346184A1360174B1B68002B03D1A2
:1020C00016481AF0B9FA1BE0134B1B6841F2E942BB
:1020D0001349184614F03AFE0346FB7397F90F3084
:1020E000002B06D097F90F3019460E481AF00AFA5D
:1020F00006E0094B1B6800220B49184614F0F8FE55
:102100001037BD4680BD00BF68DF0108540F0208CC
:1021100098DF0108BCDF010880010020DCDF010836
:10212000581B0208FCDF0108911F000880B483B02F
:1021300000AF78607B6818460C37BD4680BC70479E
:1021400080B483B000AF78607B6818460C37BD461A
:1021500080BC704780B582B000AF78607B689B68B8
:10216000002B05D07B689B687868796803229847C4
:102170007B6818460837BD4680BD80B483B000AF89
:10218000786039603A687B68134018460C37BD4662
:1021900080BC704780B500AF144B154A1A60134BD2
:1021A0004FF4E1325A60114B00229A600F4B00222B
:1021B000DA600E4B00221A610C4B0C225A610B4B59
:1021C00000229A61094B0022DA61002200210748AF
:1021D00007F0BBFB0346002B14BF01230023DBB237
:1021E000002B01D0FFF702FA00BF80BD880100205C
:1021F0000050004080B582B000AF7860786800F091
:10220000F5F800BF0837BD4680BD80B582B000AF8D
:1022100078607B681846FFF79DFF7B681846083793
:10222000BD4680BDB0B590B002AFF860B9607A60CD
:102230003B60FB68BA681A60FB687A685A60FB68A2
:102240003A689A60184BFB6200233B63FB687B6330
:1022500007F1200007F1340207F12C01134B009322
:10226000134B00F063F907F1200207F11003114648
:10227000184600F07DF907F1100540F61C0019F032
:10228000B8FE03461C462A460021204603F036FCD1
:10229000084B1C6007F110031846FFF7B6FFFB68F8
:1022A00018463837BD46B0BDF52400086F1B02083C
:1022B0006E1B0208D401002080B582B000AF7860A8
:1022C000FFF768FF074A0021074808F005FC0346AE
:1022D000064A1360786800F05BF800BF0837BD4617
:1022E00080BD00BF580F0208F5210008CC01002076
:1022F00080B584B000AFF860B9601346FB71B9686F
:10230000064800F05DF9064B1B68FA79114618463D
:1023100003F018FD00BF1037BD4680BDD00100207E
:10232000D401002080B582B000AF78600846114625
:102330001A460346FB700B46BB7013467B707B68E6
:102340001A68FB78002B01D0012300E00023194616
:102350001046FEF7DDFA7B685A68BB78002B01D087
:10236000012300E0002319461046FEF7D1FA7B68EE
:102370009A687B78002B01D0012300E000231946E6
:102380001046FEF7C5FA00BF0837BD4680BD000005
:1023900080B582B000AF786000224021084805F087
:1023A000D8FD32200AF048F901224021044805F006
:1023B000D0FD32200AF040F900BF0837BD4680BD8D
:1023C000000C014080B584B000AFF860B9601346DE
:1023D000FB80FA884FF6FF73B968034807F025FBC6
:1023E00000BF1037BD4680BD8801002080B586B093
:1023F00002AF78603A4B1B78BFF35B8FDBB203F020
:102400000103002B0CBF01230023DBB2002B15D0EE
:10241000334819F0DFFD0346002B14BF01230023CE
:10242000DBB2002B0AD04FF4007019F03FFF0346D7
:102430001A462C4B1A602A4819F0D8FD2A4B1B6803
:102440001B6803F00803082B0CBF01230023DBB239
:10245000012B0CBF01230023DBB2002B0FD0234B39
:102460001B68184603F059FC0023BB601E4B1B6819
:102470001B68BB601C4B1B685B68BB60BB681A4B6E
:102480001B681B6803F02003202B0CBF01230023D3
:10249000DBB2012B0CBF01230023DBB2002B17D0D2
:1024A0000BF0BAF90F4B196807F10E0305220092E1
:1024B0004FF400720C4807F0ECFB0C4B1B68094A08
:1024C0001168FA89184603F00BFC0BF0BFF9D6E748
:1024D000FB89B3F5007FB1D105481AF0ADF8ADE73F
:1024E000DC010020D801002088010020D401002058
:1024F00034E0010880B586B000AFF860B9601346DB
:10250000FB80094800F06AF878617B69002B06D0EF
:102510007B691B681B68FA88B9687869984700BFAF
:102520001837BD4680BD00BFD0010020F0B587B090
:1025300002AFF860B9607A603B60B86800F05BF8A1
:102540000446786800F061F80546386800F067F8DE
:102550000646B86A00F06DF80346009333462A46F3
:102560002146F86800F08DF8F8681437BD46F0BDD4
:1025700090B583B000AF786039607B681846FEF78D
:1025800083FA386800F0A6F80346002B0ED07C686A
:10259000386800F0A9F803461946204600F0AEF866
:1025A0007B68054ADA607B68044A9A607B68184653
:1025B0000C37BD4690BD00BF2127000857270008F3
:1025C00080B582B000AF78603960052239687868DC
:1025D00000F0E0F800BF0837BD4680BD80B582B08E
:1025E00000AF78600521786800F0E3F803461846EC
:1025F0000837BD4680BD80B483B000AF78607B688B
:1026000018460C37BD4680BC704780B483B000AF1D
:1026100078607B6818460C37BD4680BC704780B434
:1026200083B000AF78607B6818460C37BD4680BC2D
:10263000704780B483B000AF78607B6818460C3771
:10264000BD4680BC7047F0B585B000AFF860B9609A
:102650007A603B60FC68B868FFF7D7FF054678688A
:10266000FFF7DDFF06463868FFF7E3FF0346324613
:102670002946204600F0B5F8FB6818461437BD46D9
:10268000F0BDF0B585B000AFF860B9607A603B602E
:10269000B86800F09CF80246FB6892E8030083E803
:1026A0000300FB6803F108047868FFF7AEFF0546F6
:1026B0003868FFF7B4FF0646B86AFFF7BAFF03466B
:1026C000324629462046FFF7BEFFFB6818461437FE
:1026D000BD46F0BD80B483B000AF786001231846DA
:1026E0000C37BD4680BC704780B483B000AF7860C3
:1026F0007B6818460C37BD4680BC704790B583B0E8
:1027000000AF786039603868FFF7EEFF0346224675
:102710001946786800F0B0F800BF0C37BD4690BD90
:10272000B0B584B000AFF860B9607A60F86800F0C6
:10273000BFF80446B868FEF71CFA05467868FEF74D
:1027400022FA03461A462946204600F0BEF800BF8A
:102750001037BD46B0BD90B585B000AFF860B96028
:102760001346FB71FB79012B09D1B86800F0A0F882
:102770000446F86800F0C4F803461C6005E0FB79E5
:102780001A46B968F86800F0C7F8002318461437ED
:10279000BD4690BD80B584B000AFF860B9607A6086
:1027A0007A68B968F86800F0E2F800BF1037BD46F3
:1027B00080BD80B582B000AF7860396039687868D4
:1027C00000F0F3F8034618460837BD4680BD80B4D4
:1027D00083B000AF78607B6818460C37BD4680BC7C
:1027E000704790B585B000AFF860B9607A603B6023
:1027F0007868FFF714FF04463868FFF71AFF0346AE
:102800001A462146F86800F0E9F8FC68B868FFF756
:10281000FCFE03461946204600F0F3F8FB68184614
:102820001437BD4690BD80B582B000AF7860396086
:102830007B683A681146184600F0F4F87B68184641
:102840000837BD4680BD80B582B000AF7860396082
:102850007B683A6892E8030083E803007B6803F131
:1028600008023B68083319461046FFF7DCFF7B6817
:1028700018460837BD4680BDB0B584B000AFF860DB
:10288000B9603A71B868FFF72FFF05460C2019F0C0
:10289000B0FB03461C4629462046FFF7D4FFF868E4
:1028A00000F02EF803461C6000BF1037BD46B0BDD7
:1028B00080B582B000AF7860786800F0D6F8034643
:1028C0001B6818460837BD4680BDF0B585B000AF1F
:1028D000F860B9607A60F86800F0D3F80446B86828
:1028E000FEF747F905467868FEF74DF903462A4694
:1028F0002146304600F0CFF800BF1437BD46F0BD8A
:1029000080B582B000AF78607868FFF70FFC0346AF
:1029100018460837BD4680BDB0B584B000AFF8603A
:10292000B9601346FB71FB79032B16D0032B19DC1E
:10293000012B02D0022B0AD014E0B868FFF7B8FFD1
:102940000446F868FFF7DCFF03461C600AE02A46ED
:10295000B968F86800F0BBF804E02146F86800F0B8
:10296000D4F800BF002318461037BD46B0BD80B56F
:1029700088B000AFF860B9607A60FB68FB61BB6843
:10298000BB617B687B614FF6FF717869FFF7F5FBF0
:102990003861FB69BA69BFF35B8F1A60BFF35B8F65
:1029A00000BF00BF2037BD4680BD80B586B000AFF8
:1029B000786039607B687B613B683B614FF6FF71F3
:1029C0003869FFF7DAFBF8607B69BFF35B8F1B6840
:1029D000BFF35B8F18461837BD4680BD80B584B005
:1029E00000AFF860B9607A607968F86800F0A1F823
:1029F000B968F86800F0ABF8FB6818461037BD46B8
:102A000080BD80B582B000AF786039603868FFF76C
:102A1000FCFD03461A687B681A607B681846083715
:102A2000BD4680BD90B583B000AF7860396038682E
:102A300000F098F80346184600F09EF80346194641
:102A4000786800F0B0F87C68386800F09FF80346BA
:102A50001846FFF7DAFD034619462046FFF7D1FF77
:102A60007B6818460C37BD4690BD80B582B000AF7C
:102A700078607868FFF764FB034618460837BD4660
:102A800080BD80B483B000AF78607B6818460C3797
:102A9000BD4680BC7047B0B584B000AF3873B96034
:102AA0007A603B60B868FFF7ECFF04467868FEF791
:102AB00060F805463868FEF766F803461A46294668
:102AC000204600F092F800BF1037BD46B0BDB0B54B
:102AD00084B000AFF860B9603A71B86800F0A4F84B
:102AE00003461D680C2019F084FA03461C46234651
:102AF0002A4607CA83E80700F868FFF701FF034684
:102B00001C6000BF1037BD46B0BD80B582B000AFBD
:102B1000786039707868FFF7F3FE03461B68002B76
:102B200003D00C21184619F053FA00BF0837BD46F0
:102B300080BD80B582B000AF786039603968786850
:102B400000F07EF87B6818460837BD4680BD80B42B
:102B500083B000AF786039607B6818460C37BD469B
:102B600080BC704780B483B000AF78607B68184643
:102B70000C37BD4680BC704780B483B000AF78602E
:102B80007B6818460C37BD4680BC704780B582B064
:102B900000AF78607B68184600F05DF80346184681
:102BA0000837BD4680BD80B582B000AF786039601F
:102BB000386800F05AF80346184600F060F80346FB
:102BC0001946786800F07BF8386800F062F8034630
:102BD000184600F06AF803461946786800F085F850
:102BE0007B6818460837BD4680BDB0B586B000AFDB
:102BF000F860B9607A60B868FDF7BBFF0446786892
:102C0000FDF7C1FF024607F110032146184600F008
:102C100079F807F110032A461946F86800F089F898
:102C200000BF1837BD46B0BD80B582B000AF786038
:102C30007868FFF785FA034618460837BD4680BD19
:102C400080B483B000AF786039607B6818460C3779
:102C5000BD4680BC704780B483B000AF78607B68AD
:102C600018460C37BD4680BC704780B483B000AFB7
:102C700078607B6818460C37BD4680BC704780B4CE
:102C800083B000AF78607B6818460C37BD4680BCC7
:102C9000704780B582B000AF7860786800F080F847
:102CA000034618460837BD4680BD80B483B000AFE8
:102CB00078607B6818460C37BD4680BC704780B58D
:102CC00082B000AF78603960386800F073F803466E
:102CD000184600F07BF803461946786800F080F843
:102CE0007B6818460837BD4680BD80B582B000AF0E
:102CF000786039603868FFF7D8FF7B681846083776
:102D0000BD4680BD90B585B000AFF860B9607A600F
:102D1000B868FDF72EFF04467868FDF734FF0346D8
:102D20001A462146F86800F068F8F8681437BD467E
:102D300090BDF0B589B000AFF860B9603A71FC6839
:102D4000FB680833184600F071F8014607F11403D8
:102D5000BA68184600F077F80546FB68083318464D
:102D600000F07FF8014607F11803BA68184600F032
:102D700084F80646FB680833184600F090F80146D0
:102D800007F11C03BA68184600F095F8034632466E
:102D90002946204600F0A1F800BF2437BD46F0BD0B
:102DA00080B483B000AF78607B6818460C37BD46AE
:102DB00080BC704780B582B000AF7860786800F062
:102DC000B0F8034618460837BD4680BD80B483B0CE
:102DD00000AF78607B6818460C37BD4680BC7047F2
:102DE00080B582B000AF786039603868FFF7EEFFD9
:102DF0007B6818460837BD4680BDB0B584B000AFCB
:102E0000F860B9607A60FC68B868FDF7B2FE054604
:102E10007868FDF7B8FE03461A462946204600F0BA
:102E20008AF8FB6818461037BD46B0BD80B582B041
:102E300000AF78607B68184600F09BF803461846A0
:102E40000837BD4680BD80B584B000AFF860B9607A
:102E50007A60B86800F099F8034618461037BD4606
:102E600080BD80B582B000AF7860786800F097F8D8
:102E7000034618460837BD4680BD80B584B000AF14
:102E8000F860B9607A60786800F095F803461846F3
:102E900000F09BF8034618461037BD4680BD80B54C
:102EA00082B000AF7860786800F09FF8034618465B
:102EB0000837BD4680BD80B584B000AFF860B9600A
:102EC0007A60786800F077F80346184600F099F8C1
:102ED000034618461037BD4680BD2DE9F04186B047
:102EE00002AFF860B9607A603B60F86800F099F86A
:102EF0000446B86800F049F805467868FDF739FEE1
:102F000006463868FDF73FFE0346009333462A46DF
:102F10002146404600F08FF800BF1037BD46BDE89F
:102F2000F08180B483B000AF78607B6818460C37BE
:102F3000BD4680BC704790B585B000AFF860B96001
:102F40007A60FC687868FDF71EFE03461946204645
:102F500000F0A5F8FB681C1DB868FDF70AFE0346E3
:102F60001946204600F0AEF8FB6818461437BD46F7
:102F700090BD80B582B000AF78607868FFF706FE3C
:102F8000034618460837BD4680BD80B483B000AF05
:102F900078607B6818460C37BD4680BC704780B5AA
:102FA00082B000AF78607868FFF773FE034618467A
:102FB0000837BD4680BD80B483B000AF78607B68C1
:102FC00018460C37BD4680BC704780B582B000AF54
:102FD0007860786800F086F80346184600F08FF8AD
:102FE000034618460837BD4680BD80B582B000AFA5
:102FF00078607868FFF7DEFE034618460837BD465E
:1030000080BD80B582B000AF7860786800F081F84C
:103010000346184600F08AF8034618460837BD46AE
:1030200080BD80B483B000AF78607B6818460C37F1
:10303000BD4680BC7047F0B585B000AF3873B9604D
:103040007A603B607868FFF7A0FF03461B68BA68A8
:10305000526802F00102002A02D1BA68146808E03E
:10306000BA68526852101A441268B96809680A446A
:103070001468BA68526852109D183868FDF779FDD7
:1030800003461E68B86AFDF77EFD03461B881A4694
:1030900031462846A04700BF1437BD46F0BD90B565
:1030A00083B000AF786039607C683868FDF76BFDED
:1030B00003461946204600F043F87B6818460C3753
:1030C000BD4690BD80B582B000AF78603960386889
:1030D000FDF74FFD02467B681A607B68184608378B
:1030E000BD4680BD80B582B000AF78607B68184671
:1030F00000F036F8034618460837BD4680BD80B458
:1031000083B000AF78607B6818460C37BD4680BC42
:10311000704780B582B000AF78607B68184600F0D9
:103120002BF8034618460837BD4680BD80B483B0EF
:1031300000AF78607B6818460C37BD4680BC70478E
:1031400080B582B000AF786039603868FDF71BFD4C
:1031500002467B681A607B6818460837BD4680BD0A
:1031600080B582B000AF7860786800F011F803464F
:1031700018460837BD4680BD80B582B000AF786084
:10318000786800F013F8034618460837BD4680BD3E
:1031900080B582B000AF78607B680433184600F0D9
:1031A00012F8034618460837BD4680BD80B582B088
:1031B00000AF78607B68184600F010F803461846A8
:1031C0000837BD4680BD80B483B000AF78607B68AF
:1031D0001B6818460C37BD4680BC704780B483B06E
:1031E00000AF78607B681B6818460C37BD4680BC12
:1031F000704780B483B000AF786039607B683A680C
:103200001A6500BF0C37BD4680BC704780B584B0DE
:1032100002AF786039607B683A68DA647B680022C4
:10322000DA637B6800221A647B6800225A647B6838
:10323000002283F8392003220021012008F08DFAB2
:1032400002467B689A647B68DB6C796801221846C9
:10325000FFF74EF87B68DB6B002B45D17B681B6C5E
:10326000022B41DC7B685B6C591C7A685164D9B2D3
:1032700000230193002300930123FE22786800F0CD
:103280009BFF7B689B6C40F6B831184608F07EFDCA
:103290000346012B14BF01230023DBB2002BD9D03E
:1032A0007B685B6C591C7A685164D9B20023019326
:1032B0000023009300230022786800F07DFF7B68E4
:1032C0009B6C40F6B831184608F060FD0346012BB0
:1032D00014BF01230023DBB2002BBBD07B681B6C27
:1032E0005A1C7B681A64B5E77B6800221A647B6805
:1032F000DB6B0A2B45D17B681B6C022B41DC7B68A6
:103300005B6C591C7A685164D9B200230193002385
:1033100000930123FE22786800F04EFF7B689B6CCF
:1033200040F6B831184608F031FD0346012B14BFB2
:1033300001230023DBB2002BD9D07B685B6C591CC6
:103340007A685164D9B200230193002300930023CB
:103350000022786800F030FF7B689B6C40F6B83143
:10336000184608F013FD0346012B14BF0123002368
:10337000DBB2002BBBD07B681B6C5A1C7B681A64C9
:10338000B5E77B68DB6B472B00F39A80002BC0F21C
:103390002D81472B00F22A8101A252F823F000BFB1
:1033A000C5340008ED350008ED350008ED3500089E
:1033B000ED350008ED350008ED350008ED35000865
:1033C000ED350008ED350008C5340008ED3500087E
:1033D000ED350008ED350008ED350008ED35000845
:1033E000ED350008ED350008ED350008ED35000835
:1033F000CD340008ED350008ED350008ED35000846
:10340000ED350008ED350008ED350008ED35000814
:10341000ED350008ED350008ED3400088D35000865
:10342000ED350008ED350008ED350008ED350008F4
:10343000ED350008ED350008ED350008ED350008E4
:103440000D350008ED350008ED350008ED350008B4
:10345000ED350008ED350008ED350008ED350008C4
:10346000ED350008ED3500082D350008ED35000874
:10347000ED350008ED350008ED350008ED350008A4
:10348000ED350008ED350008ED350008ED35000894
:103490004D350008AD350008ED350008ED35000864
:1034A000ED350008ED350008ED350008ED35000874
:1034B000ED350008ED3500086D350008CD35000804
:1034C000FF2B93E07B68FF22DA638FE07B685B6C05
:1034D000591C7A685164D9B20023019300230093E8
:1034E00009230122786800F067FE7FE07B685B6C4F
:1034F000591C7A685164D9B20023019300230093C8
:1035000002230122786800F057FE6FE07B685B6C55
:10351000591C7A685164D9B20023019300230093A7
:1035200001230222786800F047FE5FE07B685B6C55
:10353000591C7A685164D9B2002301930023009387
:103540000423FE22786800F037FE4FE07B685B6C56
:10355000591C7A685164D9B2002301930023009367
:1035600008230322786800F027FE3FE07B685B6C4D
:10357000591C7A685164D9B2002301930023009347
:1035800007230322786800F017FE2FE07B685B6C4E
:10359000591C7A685164D9B2002301930023009327
:1035A00002230022786800F007FE1FE07B685B6C56
:1035B000591C7A685164D9B2002301930023009307
:1035C00010230122786800F0F7FD0FE07B685B6C48
:1035D000591C7A685164D9B20023019300230093E7
:1035E0000B230022786800F0E7FD00BF7B68DB6BEF
:1035F000FF2B09D07B689B6C40F6B831184608F069
:10360000C5FB0346012B01D0012300E00023002B62
:1036100000D1B6E600BF7B68DB6C002200211846B3
:10362000FEF766FE00BF0837BD4680BD2DE9F041BC
:1036300096B00AAFF861B9611346FB82FB69186D59
:103640004FF6FF731222B64906F0EFF9FB69186DC9
:10365000FA8A4FF6FF73B96906F0E7F9FB69186D4E
:103660004FF6FF730122AF4906F0DFF907F120039F
:103670001846FDF715F807F12002FB8A1946B869CC
:10368000FCF7ABFF034683F00103DBB2002B40F0F5
:103690002C85FB69DB6B472B00F2458501A252F8B4
:1036A00023F000BFC5370008274100082741000864
:1036B000274100082741000827410008274100084A
:1036C000274100082741000827410008333A000835
:1036D000274100082741000827410008274100082A
:1036E000274100082741000827410008274100081A
:1036F00027410008B13C0008274100082741000885
:1037000027410008274100082741000827410008F9
:10371000274100082741000827410008F93C00081C
:1037200015400008274100082741000827410008EC
:1037300027410008274100082741000827410008C9
:1037400027410008473D000827410008274100089D
:1037500027410008274100082741000827410008A9
:10376000274100082741000827410008B13D000813
:103770002741000827410008274100082741000889
:103780002741000827410008274100082741000879
:1037900027410008013F00085B400008274100085E
:1037A0002741000827410008274100082741000859
:1037B000274100082741000827410008C93F0008A9
:1037C000A740000897F82130FE2B14D197F822303B
:1037D000052B10D13B8D0C2B0DD17B6A1B78012B57
:1037E00009D17B6A01330B224F49184619F09DF924
:1037F0000346002B13D097F82130FE2B1AD197F8EF
:103800002230002B16D13B8D0B2B13D17B6A0B2260
:103810004549184619F089F90346002B0AD1FB697E
:103820000A22DA63FB69986C00230022002108F069
:10383000B3F8FDE097F82130002B14D197F822302F
:10384000042B10D13B8D0A2B0DD17B6A1B78022BE8
:1038500009D17B6A013309223449184619F065F908
:103860000346002B13D097F82130002B1AD197F87C
:103870002230002B16D13B8D092B13D17B6A0922F4
:103880002A49184619F051F90346002B0AD1FB6961
:103890000A22DA63FB69986C00230022002108F0F9
:1038A0007BF8C5E097F82130FE2B14D197F8223031
:1038B000052B10D13B8D0E2B0DD17B6A1B78012B74
:1038C00009D17B6A01330D221949184619F02DF9E7
:1038D0000346002B13D097F82130FE2B2AD197F8FE
:1038E0002230002B26D13B8D0D2B23D17B6A0D225C
:1038F0000F49184619F019F90346002B1AD1FB6934
:103900005B6C591CFA695164D9B2002301930023FE
:1039100000930223FE22F86900F04EFC88E000BF0D
:103920004CE0010860E0010864E0010870E0010873
:103930007CE0010897F82130FE2B14D197F8223053
:10394000052B10D13B8D0D2B0DD17B6A1B78012BE4
:1039500009D17B6A01330C228F49184619F0E5F82A
:103960000346002B13D097F82130FE2B1FD197F878
:103970002230002B1BD13B8D0C2B18D17B6A0C22E3
:103980008549184619F0D1F80346002B0FD1FB6981
:103990005B6C591CFA695164D9B20023019300236E
:1039A00000930223FE22F86900F006FC40E097F83D
:1039B0002130002B14D197F82230042B10D13B8DED
:1039C0000B2B0DD17B6A1B78022B09D17B6A01334B
:1039D0000A227249184619F0A8F80346002B17D09E
:1039E00097F82130002B40F0828397F82230002B8B
:1039F00040F07D833B8D0A2B40F079837B6A0A225D
:103A00006649184619F091F80346002B40F06F8381
:103A1000FB695B6C591CFA695164D9B200230193AC
:103A20000023009303230022F86900F0C5FB5EE346
:103A30005DE397F82130FE2B14D197F82230052B47
:103A400010D13B8D0C2B0DD17B6A1B78012B09D13A
:103A50007B6A01330B225249184619F066F8034677
:103A6000002B13D097F82130FE2B1FD197F822306E
:103A7000002B1BD13B8D0B2B18D17B6A0B224849A5
:103A8000184619F052F80346002B0FD1FB695B6C06
:103A9000591CFA695164D9B20023019300230093A1
:103AA0000323FE22F86900F087FB00E197F821303C
:103AB000002B14D197F82230042B10D13B8D0A2B08
:103AC0000DD17B6A1B78022B09D17B6A0133092255
:103AD0003449184619F029F80346002B13D097F8FB
:103AE0002130002B1FD197F82230002B1BD13B8DAA
:103AF000092B18D17B6A09222A49184619F015F8B2
:103B00000346002B0FD1FB695B6C591CFA695164A9
:103B1000D9B2002301930023009303230022F86904
:103B200000F04AFBC3E097F82130FE2B14D197F840
:103B30002230052B10D13B8D0E2B0DD17B6A1B78CB
:103B4000012B09D17B6A01330D221749184618F061
:103B5000ECFF0346002B13D097F82130FE2B25D124
:103B600097F82230002B21D13B8D0D2B1ED17B6A83
:103B70000D220D49184618F0D8FF0346002B15D129
:103B8000FB691422DA63FB69986C00230022002190
:103B900007F002FF8BE000BF8CE001089CE0010809
:103BA00064E0010870E001087CE0010897F821302A
:103BB000FE2B14D197F82230052B10D13B8D0D2B05
:103BC0000DD17B6A1B78012B09D17B6A01330C2252
:103BD0007449184618F0A9FF0346002B13D097F834
:103BE0002130FE2B1AD197F82230002B16D13B8DB5
:103BF0000C2B13D17B6A0C226A49184618F095FFEA
:103C00000346002B0AD1FB691422DA63FB69986C26
:103C100000230022002107F0BFFE48E097F8213082
:103C2000002B14D197F82230042B10D13B8D0B2B95
:103C30000DD17B6A1B78022B09D17B6A01330A22E2
:103C40005949184618F071FF0346002B17D097F812
:103C50002130002B40F04D8297F82230002B40F0AD
:103C600048823B8D0A2B40F044827B6A0A224E49EF
:103C7000184618F05AFF0346002B40F03A82FB69C1
:103C80001F22DA63FB6918334849184618F0C2FE50
:103C9000FB6900225A61FB69032283F83920FB6922
:103CA000986C00230022002107F076FE21E220E23A
:103CB00097F82130012B40F01E8297F82230042B18
:103CC00040F019823B8D022B40F015827B6A1B78F5
:103CD000012B40F010827B6A01331A78FB6983F86C
:103CE0003920FB691E22DA63FB69986C00230022ED
:103CF000002107F051FEFEE197F82130012B40F042
:103D0000FC8197F82230042B40F0F7813B8D0A2B81
:103D100040F0F3817B6A1B78012B40F0EE81FB6958
:103D200003F136007B6A01330322194618F0DEFAEC
:103D3000FB692822DA63FB69986C002300220021CA
:103D400007F02AFED9E197F82130022B40F0D78105
:103D500097F82230062B40F0D2813B8D042B40F0A7
:103D6000CE817B6A1B78012B40F0C9817B6A0133CD
:103D70001B781A047B6A02331B781B0213437A6A8E
:103D80000332127813431A46FB695A61FB693222E7
:103D9000DA63FB69986C00230022002107F0FCFD28
:103DA000ADE100BF8CE001089CE00108A8E001083B
:103DB00097F82130FE2B40F0AB8197F82230052B8D
:103DC00040F0A6813B8D0D2B40F0A2817B6A1B78D1
:103DD000012B40F09D81FB6903F118007B6A0133E0
:103DE0001B789C467B6A02331B789E467B6A0333B2
:103DF0001B781A467B6A04331B7819467B6A0533A5
:103E00001B781C467B6A06331B781D467B6A07338A
:103E10001B781E467B6A08331B783B617B6A09333B
:103E20001B78FB607B6A0A331B78BB607B6A0B33B1
:103E30001B787B607B6A0C331B780993D7F804806E
:103E4000CDF82080D7F80880CDF81C80D7F80C80FA
:103E5000CDF818803B69059304960395029401916F
:103E6000009273466246A74918F0D4FDFB6993F8A7
